:100000008828B400142020082104031983287D20A7
:1000100084133408800664000D280E28A00A0319F2
:10002000A10F0B2880068328FF3A841780058328B8
:10003000A000A00DA00D200D3839C1389F00003060
:10004000A100323037201F151F192428A1011E08D6
:100050008328A301A200FF30A207031CA307031CEF
:1000600083280330A100DF3037202B28A101E83E90
:10007000A000A109FC30031C4028A00703183D285C
:10008000A0076400A10F3D2820184628A01C4A287C
:1000900000004A280800A501A4011030A600210D87
:1000A000A40DA50D2208A4022308031C230FA502FA
:1000B000031861282208A40723080318230FA507A3
:1000C0000310A00DA10DA60B4F2820088328103087
:1000D000A800A101A001A70CA60C031C75282208EA
:1000E000A00723080318230FA107A10CA00CA50C3F
:1000F000A40CA80B6B2824088328A009A109A00A36
:100100000319A10A08008313031383126400080073
:1001100083169F018117FF30850007308600FF306E
:10012000870083129630BC009630BD009630BE002A
:100130009630BF009630C00086013C08A000A101A7
:1001400006308400803001203D08A000A101063067
:100150008400403001203E08A000A1010630840048
:10016000203001203F08A000A1010630840010309B
:1001700001204008A000A1010630840008300120C1
:100180003C083D07BA00BB01BB0D3E08BA07031887
:10019000BB0A3F08BA070318BB0A40083A07B80071
:1001A0003B080318013EB9003808A0003908A10037
:1001B0006430A200A3014B20C10041080F3CB800ED
:1001C0000030031CFF3EB9003908A30038082A207C
:1001D00000301820BC009630A600A7013C08A20001
:1001E000A3016720BA002508BB003A08A0003B081D
:1001F000A100FF30A200A3014B20BA002108BB00E0
:100200005A303A07BC0001301820BD009630A600D5
:10021000A7013D08A200A3016720BA002508BB0082
:100220003A08A0003B08A100FF30A200A3014B2028
:10023000BA002108BB005A303A07BD00023018202E
:10024000BE009630A600A7013E08A200A3016720C9
:10025000BA002508BB003A08A0003B08A100FF3007
:10026000A200A3014B20BA002108BB005A303A0774
:10027000BE0003301820BF009630A600A7013F083B
:10028000A200A3016720BA002508BB003A08A0001D
:100290003B08A100FF30A200A3014B20BA002108B7
:0E02A000BB005A303A07BF009C286300552966
:02400E00E13F90
:00000001FF
